:10000000F01F0010913700008D3700008D37000081
:100010008D3700008D3700008D3700000000000094
:100020000000000000000000000000008D3700000C
:100030008D370000000000008D3700002D160000F5
:10004000FD130000FD130000FD130000FD13000070
:10005000FD130000FD130000FD130000FD13000060
:10006000FD130000FD130000FD130000FD13000050
:10007000FD13000089370000893700008937000030
:10008000E5160000FD160000151700002D170000F2
:1000900089370000F5170000893700008937000014
:1000A0008937000089370000893700008937000050
:1000B0008937000089370000893700008937000040
:1000C00008B500230B60036000F006FE08BD08B50C
:1000D0000A20002101F0A6FA08BD08B5052002F0AB
:1000E000B3FE08BD38B5094B0D1C041C196801206E
:1000F00001F048FB012001F025FB291C201C02F027
:10010000CDFE012001F02EFB38BDC046C404001016
:1001100070B5054E051C0E24013C295D301C01F014
:1001200085FD002CF8D170BDC039000038B51648E7
:1001300001F07CFD154C201CFFF7EAFF144D422115
:10014000281C01F073FD201C0E30FFF7E1FF432156
:10015000281C01F06BFD201C1C30FFF7D9FF0D4857
:1001600001F064FD201C2A30FFF7D2FF281C4E212D
:1001700001F05CFD201C3830FFF7CAFF616D0648B6
:1001800001F054FD38BDC046C3390000CC04001056
:10019000C9390000D0390000D639000010B5084B2D
:1001A000041C1968012001F0EDFA012001F0CAFADF
:1001B000201C02F049FE012001F0D4FA10BDC04617
:1001C000C404001008B50020FFF7E8FF08BD0000D8
:1001D00010B5041C00F00CFC201C00210322034B72
:1001E00000F0FAFC00F00EFC10BDC0460800001044
:1001F00008B5021C0249034801F018FD08BDC046BD
:10020000EA390000E239000013B59620000201F03F
:100210002FFB1248FFF7DCFFFFF7D4FF1048FFF772
:10022000E7FF002401F0C2FB002803D001F000F832
:10023000002409E00A2001F025FA684601A9FFF729
:100240003FFF009B002B03D1064B01349C42E9DDAC
:10025000FFF7B8FF044801F0E9FC13BDEF390000D7
:10026000FE3900006F170000043A000070470000DC
:1002700000B5074B89B01A78064B68461B780649CB
:1002800001F0DFFC6846FFF7A3FF09B000BDC046E0
:10029000D0010010100000100F3A000013B5FFF756
:1002A000E7FFFFF78FFF0024684601A9FFF708FF6B
:1002B000009B002B2CD0182B21D004DC142B0DD04C
:1002C000152B20D104E0342B12D0352B1BD107E0A5
:1002D000134B00241A783E2A16D806E0104B08E08B
:1002E000104B00241A78062A0ED801321A700BE03F
:1002F0000C4B1C78002C07D0013C1C7003E0FFF76E
:1003000061FF282400E0002400F05EFBFFF7B0FF4F
:10031000C820013401F0B6F91D2CC5DD13BDC0465F
:10032000D00100101000001073B5124B041C1249CC
:10033000186803F0AFFA11490090114A114B201CC4
:1003400001F07FFC00F0AAFD002812D000F0C2FDF1
:10035000FA218900051C03F09DFA061C201C01F0FF
:10036000BDFC094B201873430849EB18321C01F0FF
:1003700068FC73BDC804001040420F001D3A000025
:10038000EA3900002A3A000018FCFFFF2E3A00006C
:1003900070B5051C0C1C161C00F02AFB291C201C27
:1003A0000022064B00F018FC301C01210922044BEE
:1003B00000F012FC00F026FB70BDC04608000010E3
:1003C0001400001010B590B0041C6846FFF7ACFF95
:1003D00069466A46201CFFF7DBFF10B010BD000025
:1003E00073B518200021FFF77DFE464E464D0024D0
:1003F0009836012001F0B6F9002C01D0002000E071
:100400000620012101F00EF9684601A9FFF758FE08
:10041000009B002B21D1002CF0D13368002B0DD094
:100420003A4B00941A6811321A6004E002F0B6FCEC
:10043000009B01330093009B102BF7DD344BED182C
:10044000DED518200021FFF74DFE2E4B94331C689B
:1004500063425C4100F080FACEE7002C06D0182BF6
:10046000C7D12C48FFF7C4FE00F0D4FA009B182B2C
:100470002BD1019B00220192822B22D004DC322B53
:100480000ED0732B20D119E0832B0FD0C22B1BD1A0
:10049000214B196801311960032916D11A6014E043
:1004A0001E4B01201B68C01A00F03AFD0120FFF727
:1004B00089FFFFF787FEFFF70AFE06E0FFF7A4FEBD
:1004C00003E0FFF7EBFE00E0019300F015FD144B95
:1004D0000120196801F056F9012001F033F9009864
:1004E000019902F0DBFC074B94331B68002B03D10E
:1004F00000F032FA012402E003F0E4F80024024D97
:1005000077E7C046CC04001020BF020000030010B3
:100510000CFEFFFF393A0000A80100102000001077
:10052000C404001013B501F009FC00F0A1FB00F0B9
:1005300071FA00200421012200F0A2FE0020021C1A
:10054000042100F0EBFE00200521012200F098FEBE
:100550000020021C052100F0E1FE1348002100F0FC
:1005600001FF0021114800F0FDFE00F027FC00F023
:100570006BFE3C24201CFFF725FF013C1E2001F0F0
:1005800081F8022CF6D101F021FC02F025FB1E239C
:1005900000930A230193064806490022064B02F005
:1005A000D5FBFFF71DFFC046984004409C40044027
:1005B00045370000C10000000003001000B500E056
:1005C00001300378202BFBD000BD00B5031C303B6D
:1005D000DAB2092A01D8181C08E020231843031CAA
:1005E000613B5738052B01D90120404200BD70B551
:1005F0000E1CFFF7E3FF0025041C06E0FFF7E5FFF4
:10060000002805DB2D010543013420780028F5D1B1
:100610003560201C70BD000008B500F05BFC011CBB
:10062000014801F003FB08BD433A000000B5C300D8
:10063000181A064BC0180723013BC25C002A03D1DD
:10064000002BF9D1012000E0002000BD680500105A
:100650007FB5194801F0EAFA00250326354219D181
:10066000281CFFF7E3FF002810D0681CFFF7DEFF0F
:1006700000280BD0A81CFFF7D9FF002806D0E81CE3
:10068000FFF7D4FF002801D004350FE00B48291CE8
:1006900001F0CCFA291C684601F0BCFB6846FFF764
:1006A00037FD074801F0C2FA6C1C251CFF2DD5DD73
:1006B000FFF73CFD7FBDC046EA3900004F3A00001D
:1006C000EE57000070B50E1CFFF778FF0D25041CD7
:1006D0002078FFF77AFF002807DB01347055013DD1
:1006E000F6D2201CFFF76AFF00E0002070BD00007A
:1006F00030B5464C87B023680868002B06D14448C3
:1007000001F094FA02F068FA012357E0012B12D1AC
:100710000379202B07D0002B05D03E49042201F09D
:10072000F0FA002803D1394B1A6801326AE03A48DE
:1007300001F07CFA5EE00378412B1BD1374C02308C
:10074000211CFFF7BFFF002854D00378422B51D162
:10075000211C02300E31FFF7B5FF00284AD0037884
:10076000432B47D1211C02301C31FFF7ABFF00287F
:1007700049D13FE04D2B23D1294D0230291CFFF7F1
:10078000A1FF002836D003784E2B33D1291C02302C
:100790000E31FFF797FF00282CD00378472B29D183
:1007A000023005A9FFF723FF059B002B22DB2A3D22
:1007B0006B651C481C4901F039FA0023236022E0D4
:1007C00005A9FFF714FF0378041C202B01D0002B90
:1007D00010D10025201C01A9FFF774FF0599041C06
:1007E000691801A801F02AFB002C03D00135042D63
:1007F000F0D108E002F0F0F90A480C4901F016FACD
:10080000024B00221A6007B030BDC046D80200106B
:10081000583A0000EA3900006E3A0000CC0400109B
:10082000F60400107A3A0000843A0000873A00008B
:1008300037B54C6824E0201CFFF7C0FE01A9FFF784
:10084000D6FE019B041C002B1DD0D8B2FF2B09DD66
:1008500000F0DEF9051C01980012C0B200F0D8F9D2
:10086000019003E000F0D4F90025019001980028E0
:1008700002D0291CFFF736FC23785A1E9341E41856
:100880002378002BD7D137BD08B5064A012113784C
:100890004B40137001D0044900E00449044801F0C2
:1008A000C5F908BDB9030010403A00008E3A0000B7
:1008B000923A000070B5051C01200821021C00F0CE
:1008C0002DFD0724012601200821002200F026FD2D
:1008D0002A1C224132400020022100F01FFD01208D
:1008E0000821021C00F01AFD013CECD270BD10B5CD
:1008F0000021041C0A1C022000F010FD201CFFF740
:10090000D9FF10BDF7B5012300930023019372B600
:100910006C46061C02AF01CC50235B421843C0B2A8
:10092000FFF7E5FF0020FFF7E2FF1020FFF7DFFFF2
:10093000E020FFF7DCFF002502200021012200F06B
:10094000EDFC705D0135FFF7B5FF842DF4D18436E1
:10095000BC42E0D162B6F7BD08B5AC20FFF7C7FFD7
:10096000AE20FFF7C4FFA520FFF7C1FF08BD38B5D3
:100970000D1C041C012200F083FC291C201C0122F8
:1009800000F0CCFC38BD08B5AF20FFF7B0FFA420C5
:10099000FFF7ADFF08BD08B5AE20FFF7A8FF08BD03
:1009A00010B5041CF820FFF7A2FF201CFFF79FFFE3
:1009B00010BD10B5041C8120FFF799FF3F20204097
:1009C000FFF795FF10BD000008B5074B20201B78EE
:1009D0001843FFF78CFF0A2000F054FE034B1878F1
:1009E000FFF7E7FF08BDC04610000010D00100105F
:1009F00008B5842202480021520001F04FF908BDD9
:100A0000BA03001008B50248FFF77CFF08BDC046D6
:100A1000BA03001008B501200821FFF7A8FF002045
:100A20000221FFF7A4FF02200021FFF7A0FF022010
:100A30000621FFF79CFF0320011CFFF798FF03200E
:100A4000011C002200F06AFC02200621002200F0B6
:100A500065FC06210122022000F060FCFFF7C8FFC0
:100A6000FFF7D0FFA220FFF742FFA020FFF73FFFD4
:100A7000C020FFF73CFF0020FFF792FF0A2000F0A4
:100A800001FE4020FFF733FF2C20FFF730FF32201C
:100A900000F0F8FD2E20FFF72AFF322000F0F2FDD3
:100AA0002F20FFF724FF0A2000F0ECFDFFF78CFF5A
:100AB000AF20FFF71CFFA420FFF719FF08BD0000BF
:100AC00000B50F290ED883280CD8CB0884225343B5
:100AD0000722C0181140044B80220A41111C1A5CE5
:100AE0001143195400BDC046BA030010F0B55B189D
:100AF000DBB216E08425CC086C4307270F40802525
:100B000004193D41EFB2A6189C4605E0064BE518D6
:100B10002B7801343B432B70B442F7DB0131634641
:100B2000C9B29942E6D3F0BDBA030010F0B589B05E
:100B3000059106921C1C5D68DB78834202D2247802
:100B4000039444E0A378234AC01A0023954209D1B4
:100B50004300181803234519039309E02A78013349
:100B60000232AD188342F9DB69782B7803910235A4
:100B7000EB1800260493019625E0082F05D1049A6E
:100B8000954224D02E7800270135F30706D5029A26
:100B9000069B0798D118C9B2FFF792FF0299761009
:100BA00001310291013707E0002202920199059A72
:100BB00008278B18DBB20793637802999942DCDB34
:100BC000019A01320192019B03998B42ECDB03985D
:100BD00009B0F0BDA13A0000F0B585B0061C0C1CB0
:100BE0000292039301F07AF800250190832708E030
:100BF000705D211C029A039BFFF798FF01302418B7
:100C00000135A74202D3019B9D42F1D305B0F0BD4F
:100C100000B50F23020918408000031F00D52833B8
:100C2000002B0EDB511E03208842804140420028E9
:100C300007D1242B06DC04218A1A0349CB18985CBF
:100C400000E0002000BDC0464E42000070B5064ED8
:100C5000051C0024A05D054B291CC018013400F0C0
:100C600081FB0A2CF6D170BD8A420000004004408E
:100C7000F8B51020FFF7EAFF094C271C1437257838
:100C80006678281C311C002200F0FAFA0234281C75
:100C9000311C012200F042FBBC42F0D1F8BDC0463D
:100CA00076420000F8B50B4C271C1437257866787F
:100CB000281C311C012200F0E3FA0234281C311CEC
:100CC000002200F02BFBBC42F0D10020FFF7BEFF5A
:100CD000F8BDC04676420000F0B589B0002404900B
:100CE0000591FFF7C5FF0220072101220694079412
:100CF00000F0C6FA02200721221C00F00FFB201C86
:100D00000B2100F0E1FAA04202D11823069301243E
:100D10000021264D03916A782F78111C0192381C0E
:100D2000012200F0ADFA381C0199002200F0F6FA19
:100D300003231F4E029314E03078717800F0C4FA58
:100D4000002807D103991B4AA3008A5C183369461F
:100D50005A500134029A039B013A013302920393E1
:100D6000023EE30F00210122A2424B41DBB28B4243
:100D700002D0029B8B42DFDA381C0199002200F07E
:100D80007FFA0199381C012200F0C8FA0A4902359D
:100D90008D42C0D1201E06D0069B049A059913608F
:100DA000079B01200B6009B0F0BDC04676420000F1
:100DB0004C4200004E4200008A42000008B501206B
:100DC000021C0B2100F05CFA01200B21002200F034
:100DD000A5FA03200221012200F052FA0320022189
:100DE000002200F09BFA08BD37B5234B10211A688A
:100DF000051C8A431A60214B8022196892010A431C
:100E00001A6001200B21002200F03AFA01200B2188
:100E1000002200F083FA1A4B9F211A68194C8A436A
:100E20001A601A6818491A60184B186802F032FDE7
:100E30008023000218432A1C20600221032000F0B6
:100E40006DFA142000F01EFC2368FF2293432360F8
:100E500023680F4A134323600E4B1A680192019ACC
:100E6000002AFADA22680C4B13402360FFF7A6FF32
:100E700001980004800D3EBD38820440808004400B
:100E80009840044000C0014000093D00C804001023
:100E9000800000012CC00140FFFFFFF810B50C4C92
:100EA0002068002813DA00202060FFF79DFF0A2841
:100EB0000ADC0120FFF798FF0138C023FF385B00F0
:100EC000984201D801232360FFF778FF206810BD06
:100ED0001C00001008B5FFF7E1FF011E08D001203B
:100EE000FFF782FF011E03D0024802F0D3FC011C71
:100EF000081C08BD50BB120008B5FFF7CFFF002843
:100F00000AD0FFF7E7FFFA22031C0021C00FD2002E
:100F10009A424841014B186008BDC046D4010010F8
:100F200010B500280DD0254B80211A688A431A601D
:100F3000234A012311681942FCD0224B03221A6074
:100F400001E0204B1860204B012200211A6019603B
:100F50001A6019681142FCD01C4B01221A601C4A0D
:100F6000802114684902214311601A1C002804D111
:100F7000124B8024196821431960164B1968884266
:100F80001AD01860002801D0134800E013481168F7
:100F900002F032FC124C2121206002F07BFC114B4C
:100FA00018609620000200F063FCFA212068890096
:100FB00002F070FC00F04CFB10BDC04638820440CB
:100FC0000C800440708004407480044078800440A9
:100FD0008080044020000010006CDC02001BB70081
:100FE000C8040010C404001008B500F03BF9134B0E
:100FF00000211A68120B12031A60114B1A68120BA7
:1010000012031A600F4B1A68120B12031A600E4B70
:101010001A68120B12031A600C4B012219600C4B58
:101020001A6019601A6019681142FCD0094B23221A
:101030001A600120FFF774FF08BDC0460080005011
:101040000080015000800250008003504080044026
:10105000448004400880044070B50F490F4800F0F8
:10106000E5FD0F4800F0E2FD0E4E0F4D00242B1958
:101070006159DA68301C0A4B143400F0D7FD782C23
:10108000F5D10A4800F0D2FD00F018FB011C084819
:1010900000F0CCFD70BDC046EA390000944200006B
:1010A000E6420000A642000024000010B142000009
:1010B000D3420000F0B53C4B8BB01D68002D3AD0F8
:1010C0003A4B02901B6801209B685DE00134237855
:1010D000202BFBD0002B3AD0B30008336A469C503B
:1010E0000136FF2D01D135E001342378202B01D0CA
:1010F000002BF9D1202B02D1002323700134012EC3
:101100001BD12A4F2A4B07223B6001923D1C09E06C
:101110002B680298196800F003FE002808D02B689D
:1011200014332B60019B013B0193002BF0D132E083
:101130003B681D7901E0041C2E1C2378002B06D08F
:1011400000230722B2425B41DBB2002BBFD1002E4D
:101150001CD000E00025154C022E05D1039815493E
:1011600000F0DEFD002801D0AE420AD82368124804
:10117000D96800F05BFD23681048196900F056FD3E
:1011800004E02368F0B29B6802A99847064B1B68ED
:10119000002B07D103E00198011CFFF75DFF084811
:1011A00000F044FD0BB0F0BDD8020010E0020010CA
:1011B00024000010E0420000E24200007F3A0000FC
:1011C000E942000038B5041C154D0A2808D002D8A1
:1011D00008281CD110E00D2802D07F2817D10BE081
:1011E0002B6800221A700F4800F020FD0E4C201CC6
:1011F000FFF760FF2C6012E02A680B4B9A420ED971
:101200000A48211C00F012FD2B68013B06E007484C
:10121000211C00F00BFD2B681C7001332B6038BDC6
:10122000DC020010E6420000D8010010F542000088
:1012300008B503E000F098FBFFF7C4FF00F0B6FB31
:101240000028F7D108BD000008B5034A034B044845
:101250001A6000F0EBFC08BDD8010010DC020010A1
:10126000E9420000044B40211A680A431A60034B0C
:1012700001221A707047C04680800440E4020010CA
:1012800070B50E4B061C1B780D1C141C002B01D1D5
:10129000FFF7E8FF013E022E03D8094BB600F358D2
:1012A00000E0084B1A68012C03D1AC4014431C60C9
:1012B00003E00124AC40A2431A6070BDE4020010B8
:1012C000784300000080005038B50F4B051C1B7898
:1012D0000C1C002B01D1FFF7C5FF0020032D11D8F6
:1012E000281C012302F074FA02040608074A04E0ED
:1012F000074A02E0074A00E0074A1068A340184086
:10130000431E984138BDC046E4020010FC3F005027
:10131000FC3F0150FC3F0250FC3F035070B50E4BA8
:10132000061C1B780D1C141C002B01D1FFF79AFF23
:10133000013E022E03D8094BB600F35800E0084BDB
:101340001A68012C03D1AC4014431C6003E0012453
:10135000AC40A2431A6070BDE40200108443000058
:10136000FC3F005038B5084B041C1B780D1C002BAB
:1013700001D1FFF777FF2368182293432360236886
:101380001D43256038BDC046E40200101F234209FA
:10139000184001238340181C014B9200D050704725
:1013A00000E100E01F234209184001238340181C7C
:1013B0002032024B9200D0507047C04600E100E05E
:1013C000054B3F221A60054B01221A60044B402155
:1013D0001A688A431A60704724800440D880044009
:1013E0003882044008B5044B40211A688A431A60C9
:1013F000FFF7E6FF08BDC0463882044008B5154B2C
:101400001868FFF78DFD0720FFF7CCFF0820FFF7D6
:10141000C9FF0A20FFF7C6FF0C20FFF7C3FF0B2010
:10142000FFF7C0FF0920FFF7BDFF0B4A0023136041
:1014300001210A4A49421160094A1360094A1360AE
:10144000094B01221A60094B1A6801321A60C04622
:1014500008BDC046200000100482044008820440F9
:1014600004C000403CC0004000C00040E802001042
:1014700008B5FFF717FC0A480021FFF773FF09487A
:101480000021FFF76FFF08480021FFF76BFF0748B7
:101490000021FFF767FF06480021FFF763FF08BD43
:1014A0000840044000400440AC4004401440044064
:1014B0001C400440F8B5071C0C1C72B6FFF7D8FF9F
:1014C000434B1A68434B1A60002F01D0424B00E097
:1014D000424B434A04211360424B434D1A680A436E
:1014E0001A6000232B609C4218D00720FFF74EFFA4
:1014F0000820FFF74BFF0A20FFF748FF0C20FFF7FB
:1015000045FF0B20FFF742FF384B394A19680A4064
:101510001A602A68EC235B0113432B60002F4FD025
:10152000344B354C354900260E60201C1E60311CA2
:10153000FFF718FF301C0921321CFFF7A1FE301CF9
:101540000921321CFFF7EAFE2D4B80221968114356
:101550001960236807218B432360236802210B4312
:1015600023607B00DB1999015B189B002549DF197B
:10157000254B0F6003211960244B25491868014051
:101580001960196809200A431A60FFF7FFFE174A1D
:10159000802311689B00194311602A6802211343BC
:1015A0001C4A2B60012313601B4A11601B4A13491C
:1015B00013601660136010681842FCD001230B60A2
:1015C000174B012252421A6062B630BFF8BDC046C6
:1015D0003882044034820440BF180000FF18000025
:1015E0003082044010ED00E0048204400082044098
:1015F0007FE2FFFF044001406440044004C000401B
:101600008080044018C0004014C000403CC000402E
:101610000FF0FFFF78800440708004407480044025
:101620000882044008B5FFF745FF08BD00B5064B2A
:101630001A6801321A601B68013303D1034B1A6820
:1016400001321A6000BDC046F0020010EC0200102A
:1016500000B5074B98420AD8064A00231360064A91
:1016600001381060054A1360054B07221A6000BD5F
:10167000FFFFFF00F002001014E000E018E000E0BF
:1016800010E000E000B50C4A1368002800D10120EA
:10169000C1438B4204D809E011688142FCD301E0C8
:1016A000591C081811689942F6D203E01168C91A4A
:1016B0008142FBD300BDC046F002001010B5064BBE
:1016C000FA211868054B89001C6802F095F8044B54
:1016D0005C43201810BDC046F0020010EC02001060
:1016E00037894100034B01221A60034B1A6801320B
:1016F0001A60704700C00040F4020010034B012242
:101700001A60034B1A6801321A60704700000140EA
:10171000F8020010034B01221A60034B1A680132D1
:101720001A60704700400140FC020010034B012288
:101730001A60034B1A6801321A607047008001403A
:101740000003001000B5002803D1044B01221A60E9
:1017500003E0012801D1024B186000BD04400140A4
:101760000480014000B5002802D1044B186004E059
:10177000012802D1024B00221A6000BD0440014042
:101780000480014010B500280FD1124B80221C6844
:10179000920022431A60104B032218600F4B19600D
:1017A0000F4B1A608022D20211E0012811D1094B9F
:1017B00080221868D20002431A600A4B00221A6085
:1017C000094B03221960094B1A6080221203084B4F
:1017D0001A6010BD80800440FC02001018400140D7
:1017E00014400140000300101880014014800140A3
:1017F00000E100E008B5184B1A680E231340062BD1
:101800000DD1164B9E221B68DBB2134204D0144A42
:101810005360144B1B681EE0D9071CD501E0042B54
:1018200005D1104B1868C0B200F0AFF813E00C2BD4
:1018300006D10B4B8022596852000A435A600AE0D5
:10184000022B08D1054B1A68054B910601D50022E1
:1018500000E001229A6008BD08800040148000402A
:10186000040300100080004000487047040300108B
:1018700070B5294C294B80229203DA67061C00219F
:10188000201C902200F00AFA0023A360244B0725B5
:101890001A68244CAA431A6019680122114319607E
:1018A000214B1968A94319601968114319601F4B2E
:1018B000802118684901014319601D4B1A60832279
:1018C000226019681B4B186801F096FF311C000953
:1018D00001F092FF1849030A184A0B60C0B20323B3
:1018E00010602360164B1D60164B186860201C6842
:1018F0000440602CFBD101E0146800E001201C686A
:101900000442F9D1044B01221A700F4B802292033A
:101910001A6005230B6070BD0403001004E100E0B1
:10192000A44004400C800040A84004408080044053
:1019300098800440C80400100480004000800040EB
:10194000088000401480004000E100E000B5044A37
:10195000202311681942FCD0024B186000BDC0461C
:10196000148000400080004008B5FFF77DFF827BB7
:10197000031C8218D07B9A7B0132D2B29A7352B286
:10198000002A01DA00229A7308BD10B5041CFFF783
:101990006BFF437BC318DC73437B0133DBB24373C0
:1019A0005BB2002B01DA0023437310BD08B5FFF7CB
:1019B0005BFF827B437BD01A431E984108BD30B544
:1019C000002402E00570013401301D5D002DF9D1C5
:1019D000121B131C02E00170013B0130002BFADCEA
:1019E000D043C0170240A01830BDF8B5051C0F1C2D
:1019F0001E1C541E092B01D800240FE0181C0A21BC
:101A000001F0FAFE221C031C391C281CFFF7EDFF15
:101A1000041C2D1805E02F7001340135013A002A0D
:101A2000F9DC301C0A2101F02BFF30312970601CD9
:101A3000F8BDF8B50C1CD9175F18061C4F40551E91
:101A4000092F12D9381C0A21002B03DA01F0D4FE29
:101A5000434202E001F0D0FE031C211C2A1C301C72
:101A6000FFF7E7FF041C351813E0002B00DA951E82
:101A7000002201E0B4540132A91A0029FADCEC4337
:101A8000E4172C403519002B03DA2D232B70013479
:101A90000135381C0A2101F0F3FE30312970601C39
:101AA000F8BD73B5069E041C1D1C3009531E00288A
:101AB0000AD000901A1C201C2B1CFFF7F2FF2418E0
:101AC00005E0217001300134013A002AF9DC0F23CE
:101AD0001E40092E01D8303604E0002D01D03736E3
:101AE00000E057362670013076BDF0B585B0041C95
:101AF0000F1C002801D00021017000256BE0252972
:101B000003D021700132013405E05178252904D138
:101B100021700232013401355DE0302903D00132F9
:101B20000292202101E002320292029E9C4632780B
:101B30002D3A50424241B6180296002205E00A238F
:101B40005A438218303AD2B201363078031C303B07
:101B5000092BF4D90296AE186346BE4201D97A1B0E
:101B6000D2B269280ED006D863282CD0642809D0B8
:101B700058283ED119E075280AD078280FD073284C
:101B800037D11AE01E1D201C1B68FFF752FF04E02E
:101B90001E1D201C1B68FFF728FF331C17E01E1DAD
:101BA0001B68201C0093002304E01E1D1B68201CE2
:101BB00000930123FFF775FFEFE71E1D201C1B6834
:101BC000FFF7FDFEE9E71A68012022700433029A4C
:101BD000241801322D181178BD4201D200298ED16E
:101BE0000023BD4201D2237005E0013C2370013D7A
:101BF00001E001256D4205B0281CF0BD10B50C1C9C
:101C0000131C6421221CFFF770FF10BD00B5031CDC
:101C10009BB00A1C01A8191CFFF7F0FF632800DD28
:101C2000FEE701A800F0A6F81BB000BD0FB407B591
:101C300004A901C90191FFF7E9FF03B008BC04B092
:101C400018470EB403B503AA02CA0192FFF7D6FFE4
:101C500002B008BC03B0184770B50323041C184237
:101C600005D10D1C041C194201D1934201D300235C
:101C700011E0131C40CD043B40C4032BFAD8141FC1
:101C8000A4080134A400032309191A400419EEE73B
:101C9000CD5CE55401339342FAD170BD30B50B04ED
:101CA0000D061D430D430B021D430323041C9342E9
:101CB0000DD218420BD1131C043B20C4032BFBD8BC
:101CC000141FA4080134A40003231A40041900239C
:101CD00001E0E15401339342FBD130BD00B5002354
:101CE00000E00133C25C002AFBD1181C00BD00B526
:101CF000031C01E0013101330A781A70002AF9D17E
:101D000000BD30B5031C002406E01D5D085D281AE7
:101D100005D10134002D02D09442F6D1002030BD0F
:101D200000B502E00130002B06D00A7803780131BB
:101D30009342F7D0981A00E0181C00BD08B5FFF7D1
:101D400053F90B4BFA211868890001F0A3FDFFF746
:101D50007FFCFFF787FAFFF745FB96200002FFF7AD
:101D600087FDFEF757FEFEF743FEFFF76DFA08BD4D
:101D7000C804001010B5041C02E00134FFF7E6FDB2
:101D800020780028F9D110BD30B5F8238A01DB0096
:101D900013404A05920E1343F822120211401943D0
:101DA0000A235943CA1083181C1CEB345D7824782D
:101DB000EA336C401B7824021C43835C201C58408F
:101DC0000723194008418005800D30BD7047000091
:101DD00008B5054B011C984201DD044BC1180448AD
:101DE000EA38FFF7D1FF08BDFF17000000F8FFFF3A
:101DF0009043000008B54018511A013101F0ACFDC4
:101E000008BD08B5801889189A1A0132FFF724FF17
:101E100008BD000010B5CB00591A074B0F22C91896
:101E20000023CC5C14400470CC5C01332409447062
:101E30000230072BF5D110BD6805001010B5CB009E
:101E4000591A064BC918002342780478120122431C
:101E5000CA5401330230072BF6D110BD68050010BB
:101E600030B5B14B87B0D96EB04D4A1E91416A462C
:101E7000D175A96A1A1CC806400F0138062807D870
:101E800001F0A6FC040C1F1217191C00022409E023
:101E90005A6E16329200D3581C1C15E05B6E163336
:101EA0009B00D45800230FE09B6DD46DA3420ADC45
:101EB0000AE0022403E00C24032305E00D24231C84
:101EC00002E00D24EEE70D242C6148111F2800D9F3
:101ED00022E16A461732944901F084FC2000220076
:101EE00028002A002D002F0038004000440049003F
:101EF00051005F0067006F00770085009300A2002B
:101F0000B400C300D500D300E300E600E900F1000F
:101F1000010105010F01110113011901081C00E065
:101F20008348191C221CFFF765FFF5E08148F8E79C
:101F30000A1C0E3203E07E4809E00A1C1C32081C11
:101F4000111C1A1C231C01F077F8E5E07948011CEC
:101F50000E391A1C231CFFF754FFDDE07448011CE6
:101F60000E31EEE70A1C1C32081C111CF1E70A6E48
:101F70001020002A00D00A200A1C0E3206E00A6E49
:101F80001020002A00D00A200A1C1C3200946C4643
:101F9000173402900194081C51E001201070086E63
:101FA0001022002844D00A2242E00A6E1020002AA3
:101FB00000D00A200A1C0E320EE001201070086EBC
:101FC0001022002855D00A2253E00A6E1020002A61
:101FD00000D00A200A1C1C3200946C461734029070
:101FE0000194081C78E00A6E1021002A00D00A2112
:101FF000504A68461730019002910094101C111C41
:102000001DE00A6E1020002A00D00A20494A0094E0
:102010006C46111C173402901C390194101C0EE000
:10202000096E012010701022002900D00A224149B7
:1020300068461730019002920094081C002201F0BB
:1020400005F869E00A6E1020002A00D00A20394AFB
:1020500000946C46111C173402901C390194101C1A
:102060003AE0096E012010701022002900D00A22E7
:10207000304968461730019002920094081C0022F3
:102080002AE0012010700A6E1021002A00D00A21D7
:10209000284A68461730019002910094101C0021D4
:1020A0001AE0009222481CE00092224819E00A6ED1
:1020B0001020002A00D00A200A1C1C3206E00A6EFA
:1020C0001020002A00D00A200A1C0E3200946C4610
:1020D000173402900194002000F0E1FF1CE0009210
:1020E000081C002104E00D1C1C35081C0092291C52
:1020F0001A1C231C01F02EF80EE0081C02E00C480C
:1021000000E00C48191C221C01F03DF804E0081CFA
:10211000221C191C01F042F86B46DA7D024B07B015
:102120000120DA6630BDC046CC040010680C0010F7
:10213000DA040010E804001010B506490B1C8833BF
:102140001A68141C1E34A4006050013203210A4096
:102150001A6010BDCC040010054B0320191C8831F7
:102160000A68013A02400A601E329200D058704755
:10217000CC040010F8B5114D2C1C8C3420680130B3
:10218000FFF726FE0E4B0122D8629F6AAB6E061C3B
:1021900002409A4210D1830703D420680230FFF72F
:1021A000CBFFFF239B001E40B601BF10044B8C35B4
:1021B000374301222F60DA600220F8BDCC04001002
:1021C000680C001030B50C4B0C489A6A031C8C3319
:1021D0001C68D3059B0E910500D5403B856E92107F
:1021E00001210A40AA4204D1E3188C300360024B5B
:1021F000D960012030BDC046680C0010CC0400102E
:1022000008B5084B5A1CD07F9A1CD27F00011202DD
:102210001043DA7F0333DB7F10431B031843FFF7C0
:102220008BFF08BDCC04001038B5FFF795FF0649B9
:1022300003230F22051C5C1815400133257700117C
:10224000072BF7D138BDC046CC04001008B5FFF706
:1022500083FF034B01228C331860024BDA6008BD08
:10226000CC040010680C001010B5064CA36E002BB7
:1022700006D0FFF771FF044B8C3401222060DA6036
:1022800010BDC046CC040010680C001010B5064C00
:10229000A36E002B06D1FFF75FFF044B8C340122A5
:1022A0002060DA6010BDC046CC040010680C00103D
:1022B00008B5124B1B68002B00D09847104B5A6989
:1022C000002A15DD012A07D1DA69002A04D09A61B3
:1022D0000022DA610A225A615B690322191C9143C8
:1022E0000A1E02D0074A0121D166054A013B53610B
:1022F000044B90331A68024B5A6208BD94030010D5
:10230000680C0010CC04001000B5064B5A69002A76
:1023100007DD9A690F21044B1140D977121101335F
:10232000DA7700BD680C0010CC040010044B597F14
:102330009A7F090112020A43197F0A435A677047BC
:10234000CC04001030B50B1C093B012B0FD8084AF8
:1023500000239C18257FC45CA54205D0054B083995
:102360005A681143596002E001330E2BF1D130BDA0
:10237000CC040010680C001008B508290DD01929EC
:1023800013D1427808231A4202D00022027002E0E0
:102390000F2303700723437005E000231A1CC25467
:1023A00001330E2BFBD1FFF749FD08BD1FB50E4BC6
:1023B0005C6F002802D00F22944304435C67FF2C1B
:1023C00010DC6846211CFFF725FD6846211CFFF73D
:1023D000D3FF054A00236C46185D9918013308772E
:1023E0000E2BF8D11FBDC046CC04001030B5124CE6
:1023F0000F23656F85B09D4305436567082D19D090
:10240000FF2D17DC6846291CFFF704FD6846291CD0
:10241000FFF798FF00231A19127F69465A540133B7
:102420000E2BF8D16846291CFFF7A6FF6846291C29
:10243000FFF704FD05B030BDCC0400101FB50F4CF4
:10244000616F082918D0FF2916DC6846FFF7E2FC07
:10245000616F6846FFF776FF00231A19127F6946FD
:102460005A5401330E2BF8D1616F6846FFF784FF91
:10247000616F6846FFF7E2FC1FBDC046CC04001048
:1024800010B50D4C631CD87FA31CDB7F00011B0221
:102490001843E37F1843E31CDB7F1B031843FFF75C
:1024A00097FC0F23021C1A402277021113400012DE
:1024B0006377A07710BDC046CC040010044B5A6E61
:1024C00016329200D258121A51424A41DA667047C7
:1024D000CC04001000B5064B5A6E16329200D1584B
:1024E0000139D150002901DA0D21D15000BDC0467B
:1024F000CC04001000B5064B5A6E16329200D1582B
:102500000131D1500E2901D10021D15000BDC0466A
:10251000CC04001000B5094B5A6E16329200D25806
:102520000D2A03D11A1C2932127805E09A18507F1F
:10253000117F0001021C0A435A6500BDCC04001043
:1025400010B5084B0F245A6E16329200D1585A6DAE
:1025500058181440013104770D2902DC5B18121160
:102560001A7710BDCC04001030B50F4B5A6E596D60
:1025700016329200D2580D2A07D11C1C2934247817
:10258000F02008402043586507E09818447F057FF5
:1025900024012C435C650B114377034B9A180F23DE
:1025A0001940117730BDC046CC04001008B504486E
:1025B0000022011C1C390D23FFF723FC08BDC04677
:1025C0000405001008B504480022011C1C310D232D
:1025D000FFF717FC08BDC046E804001008B5044822
:1025E0000022011C1C310D2300F026FD08BDC04651
:1025F000E804001008B504480022011C0E390D2320
:10260000FFF7FFFB08BDC046F604001008B50448FC
:102610000022011C0E310D23FFF7F3FB08BDC0465D
:10262000E804001008B504480022011C0E310D23F7
:1026300000F002FD08BDC046E80400100C4A00236B
:10264000111C46310B70111C47310B70111C4831A5
:102650000B70111C49310B70111C4A310B70111C8D
:102660004B310B70111C4C314D320B701370704795
:10267000CC04001000B5074A011C042300208A186E
:1026800004E0D1184631097840000843013BF8D2F4
:1026900000BDC046CC04001030B5074A002389189D
:1026A000012206E0CC18051C463415402570401068
:1026B0000133042BF6D130BDCC04001038B5002016
:1026C000FFF7D8FF084C051C0021207FFFF7E4FF2F
:1026D00025770420FFF7CEFF0421051C607FFFF75C
:1026E000DBFF657738BDC046CC04001010B5002074
:1026F000FFF7C0FF034C20770420FFF7BBFF607794
:1027000010BDC046CC04001010B5054C0021207F40
:10271000FFF7C2FF607F0421FFF7BEFF10BDC04678
:10272000CC04001010B5094C231C8C331868013000
:10273000FFF74EFB064B021CD8620F231A4022778C
:102740000211134000126377A07710BDCC04001073
:10275000680C001010B5094C0021201C0D22FFF759
:1027600049FB201C0E3000210D22FFF743FB201CEB
:102770001C3000210D22FFF73DFB10BDCC040010E2
:1027800010B50C4B00211A1C187F1C780131204316
:10279000187701330E29F7D1936E002B08D0064B22
:1027A0001B690D2B04D1137F111C29310B7053733E
:1027B00010BDC046CC040010680C001010B50C4BC6
:1027C00000211A1C1C7F1878013120401877013332
:1027D0000E29F7D1936E002B08D0064B1B690D2BE9
:1027E00004D1137F111C29310B70537310BDC046E7
:1027F000CC040010680C00107FB500230C4A0D2596
:102800001C1C1118097F01306E469955C60F854270
:10281000664176420133111C30400E2BF1D100236A
:102820006C46185DCA18013310770E2BF8D17FBDA6
:10283000CC04001010B5074B5A6E16329200D158D6
:102840005C1801392077D150002901DA0D21D150CF
:1028500010BDC046CC040010034A0023111C943163
:1028600098320B6013607047CC040010034B0121B9
:1028700094331A684A401A607047C046CC0400106E
:10288000044A002313678C321360034B0122DA6081
:102890007047C046CC040010680C001008B59A4B75
:1028A0000F20996A994A8B101840891101385256A5
:1028B0000E2800D9C1E000F08BFF08111A2327C0B1
:1028C0002EC0C037C0C0C03B3F00002A00DAB4E0D1
:1028D0008F4B9A18403200239371A9E0002A00DA46
:1028E000ABE08B4B01209A1840329071A4E0002A93
:1028F00000DAA2E0864B9A1840329279DA6697E0C5
:10290000081CFFF797FF93E0002A00DA95E0101CFF
:10291000FFF7D4FD8CE0002A00DA8EE07C4B596E84
:1029200016318900CA5083E0081CFFF75FFD7FE085
:10293000081CFFF73BFD7BE0002A00DA7DE0101C5D
:10294000FFF75AFF74E0724B01209833186073E070
:10295000FFF7E0FD6CE0FFF793FF69E0FFF726FE6D
:1029600066E0FFF7EDFD63E0694B00225A665FE029
:10297000FFF728FE5CE0FFF7F7FD59E0644B01200C
:10298000586659E0FFF72AFE52E0FFF7CBFE02201F
:1029900052E0FFF72FFE4BE0FFF732FC48E0FFF775
:1029A00035FE45E0FFF7D6FE42E0FFF73DFC3FE095
:1029B000FFF738FE3CE0FFF7A7FC39E0544B00225C
:1029C0001A6635E0FFF7B2FC32E0514B0120186681
:1029D00032E0FFF741FF2BE0FFF730FD28E0FFF783
:1029E00045FF25E0FFF74CFD22E0FFF78DFE1FE0DD
:1029F000FFF73AFC1CE0FFF7C3FE19E0FFF776FE95
:102A000016E0FFF743FC13E0FFF7D8FE10E0FFF7F6
:102A100015FE0DE0FFF74CFC0AE0FFF75BFD07E059
:102A2000FFF74CFE04E0FFF765FD01E0FFF70EFC49
:102A3000012001E00120404208BD982BBED03EDCC1
:102A4000382B9BD01DDC1C2B00D187E70CDC0C2B1A
:102A500000D178E702DC002BEAD0EBE7162B00D19F
:102A600076E7182BE6D176E7282B00D17CE702DC4D
:102A7000262BDFD175E72C2B00D179E7362BD9D166
:102A800079E7662B00D18AE70CDC4C2B00D17CE780
:102A900002DC3C2BCED175E7562B00D179E75C2BBD
:102AA000C8D179E76C2B00D17FE702DC682BC1D15C
:102AB00078E7762B00D17BE7882BBBD17BE7E62B31
:102AC00000D19BE726DCC82B00D188E70CDCA82BC3
:102AD00000D17AE702DC9C2BACD173E7B82B00D194
:102AE00077E7BC2BA6D177E7D62B00D17DE703DCB7
:102AF000CC2B00D09EE775E7D82B00D178E7DC2BF4
:102B000000D097E777E7C046680C001090570000A8
:102B1000CC040010F32B00D17CE70EDCEC2B00D1B1
:102B200072E703DCE82B00D084E76AE7F12B00D1E1
:102B30006DE7F22B00D07DE77AE7F62B00D16FE747
:102B400003DCF52B00D075E767E7F72B00D16AE7C8
:102B5000F82B00D06EE769E738B5184C231C8C338E
:102B60001868FFF735F9E26E154BA2660022E2669F
:102B7000DA6003229862251C10401C1C022809D030
:102B800090420AD0012802D0FFF788FE07E0FFF745
:102B9000F1FA04E0FFF764F901E0FFF713FB002806
:102BA00007DDE368002B04D12B1C8C331A68121844
:102BB0001A6090352B681B182B6038BDCC040010B0
:102BC000680C0010034B0122DA660F229A775A77BD
:102BD0001A777047CC04001010B5054C0549201C2D
:102BE00000F0BAFEFFF7EEFF0123636610BDC0469A
:102BF000CC0400109C07000000B5074B00201B68A8
:102C00000F2B08D1054B1A78824204D11868044B67
:102C10001840431E984100BD9C000010CC040010D9
:102C200000FFFF0038B5164B1A1C98321268002AB4
:102C300004D0144B1D6801231D4001E094331D682E
:102C4000114CA3689D4202D16268002A16D0002D63
:102C500002D1002B0AD111E00C4B1B68002B02D0D3
:102C60006168281C98470023636006E0074B1B68D7
:102C7000002B02D0281C291C9847A56038BDC046EF
:102C8000CC040010B4030010680C0010AC0300105A
:102C900013B5002300930193244B1B68002B02D033
:102CA000684601A998472249009B0878214A0028D4
:102CB0000CD0002B02D00223137035E01378013BB7
:102CC000DBB21370002B2FD10B7009E0002B0CD15D
:102CD0001378002B28D0013BDBB21370002B23D1DB
:102CE000154A1360154A13601EE014490968581A02
:102CF000444260414000107011484469021C002C9D
:102D000004D08B4202D10A2343610DE000290BD18C
:102D10000A21516101999361D161084A1360064B00
:102D200002221960034B1A7013BDC0469C030010A9
:102D3000B8030010A00300109C0C0010980C0010A9
:102D4000680C001008B5FFF7A3FF08BD30B50A4DA9
:102D5000049C28600948016009490A60094A136017
:102D6000094B039A1A60094B094A1C60094B1C6005
:102D7000094B1A6030BDC046AC0300109C03001024
:102D8000A8030010A4030010980300109C0000107A
:102D9000452D0000680C00109403001008B5084B86
:102DA000084A196812688A1A1A6006D5FA2252006F
:102DB0001A60054B1A6801321A60FFF733FF08BD2D
:102DC000A000001098030010B4030010F7B50E1C0B
:102DD0000E21051C019200F0BFFD1A4B03240C27A5
:102DE0009E420FDD09236B7301232B7328E0301CF7
:102DF0000A2100F0A5FD301C29550A2100F04AFDEA
:102E00000134061C002E06D0E30F0022A7425341D6
:102E1000DBB29342EBD1019AA31A033B2B70621BE6
:102E20002B1C01E0195D5973013BD1180229F9D11E
:102E30000F231C1B002301E0013C2B55032CFBDC62
:102E4000F7BDC046FFC99A3BF8B5104B01221A7076
:102E50000F4B0222041C1A700E4E0F4D0FE0196822
:102E600091420FD01B682B60FFF798FFFFF710FF10
:102E7000002C04D0013C002C01D13C7005E03368EB
:102E80002A68024F39780029E9D1F8BDB80300104B
:102E9000A0030010A4030010B003001070B52A4B6B
:102EA0002A4C1A1C94321268A061E161002A17D1E1
:102EB00018280BD1C32909D1254A12680F2A05D138
:102EC000181C38300E21162200F0A2F8A369182B26
:102ED00004D1E369332B01D100F044F8FFF772FE0F
:102EE0000A236361184C0123251C23678C35FFF7E7
:102EF00033FE002801DAFDF7B9F92B68154A934231
:102F000003D0154A934209D104E0FFF78BFEFDF789
:102F1000E4F803E0FFF786FEFDF7D9F80F4B1A68D7
:102F20000F4B10681968884205D012681A60FFF7C5
:102F300035FFFFF7ADFE266F002ED8D1FFF772FEEA
:102F4000301CFFF781FF70BDCC040010680C00102E
:102F50009C000010F7050000070C0000A4030010FF
:102F6000B003001070B5254C002023681D68FFF7E2
:102F70006BFF23681A689542FCD01E68FFF722FE9B
:102F80001F4B0A221F4C5A6118229A611522DA61DE
:102F9000231C903300221A60FFF714FE2D36012304
:102FA0002367FF36154C184D0AE0FFF7D5FD23685F
:102FB0002A681968914203D01B682B60FFF7EEFE68
:102FC00023681B689E42F0D10E4C1820231C9033BE
:102FD00000211D68FFF762FF0C4B281C196800F0E8
:102FE00059FC3834011C0422201CFFF7EFFE044B6F
:102FF00018229A610022281CDA6170BDA403001017
:10300000680C0010CC040010B003001098030010EE
:10301000F0B501240DE005780B1C254006E0C65CE8
:10302000ED0077083D43C554351C2540013BF6D5DE
:10303000013A002AEFDCF0BD30B504E0845C8D5C21
:1030400085548C5401329A42F8DD30BDF7B5099DA4
:103050000AAC2678089F2C7894461D1C002A0DD1B6
:1030600018E063465B5D4A5DD21813190192002493
:10307000B34201DB9B1B012443550135BD42F0DD0A
:103080000AE0CA5C12190024B24201DB921B01243F
:10309000C2540133BB42F4DD099B1C70F7BDF7B588
:1030A000099E0AAC2778089D347800282FD0002983
:1030B0002AD01E1C9446002A0ED1013F18E0634618
:1030C0009B5D8A5DD21A131B00240192A34201DA90
:1030D000DB19012483550136AE42F0DD37E0CA5CCE
:1030E000121B0024561C01D13A1C0124C254013386
:1030F000AB42F4DD2BE0D15C49420C1B211E01D018
:10310000E1190124C1540133AB42F4DD1FE0002971
:103110001BD0181C002A06D10EE00E5C135C013097
:10312000F31A1C1BE40FA842F7DD10E0CA5C013360
:10313000141B013462425441AB42F7DD07E0D15C1D
:10314000013349420C1B611E8C41AB42F7DD099AE9
:103150001470F7BD70B5049D01242C70141C002957
:1031600005D10BE0065D0A5D96420BD101349C420D
:10317000F8DD05E0815C002904D101329A42F9DDD5
:1031800000232B7070BD00B503E043185B784354F7
:1031900001319142F9DB0023435400BD00B504E046
:1031A0008318013B1B788354013A8A42F8DC0023E0
:1031B000835400BDF0B5114B1A785B78825C1A40DD
:1031C00000D040220E4C0F49231C261C04C32C3671
:1031D00000221A6001240A1C123117785578C75D45
:1031E0003D4202D01F6827431F60023264008A42BA
:1031F000F3D10433B342EBD10020F0BD99010010AC
:10320000300E0010E500001030B512234B43334A56
:103210000131D3188A0051181A785C78825C144204
:1032200004D02F4A5F245218947054709A78DC7836
:10323000825C144204D02A4A7C24521853321470FF
:103240001A795C79825C144204D0254A7C24521895
:10325000A33214709A79DC79825C144207D0204C36
:103260005F226418251CA235A1342A7022701A7AB4
:103270005C7A825C144204D0194A7C245218A03231
:1032800014709A7ADC7A825C144204D0144A7C244A
:103290005218503214701A7B5C7B825C144207D047
:1032A0000F4C5F226418251C523551342A7022704D
:1032B0009A7BDC7B825C144204D0094A2E2452188B
:1032C000A43214701A7C5B7C825C134204D0044BE1
:1032D0005918F43127230B70002030BDE500001091
:1032E000A00C0010F8B52D4C071C0025201C202137
:1032F0004F22FEF7D3FC002D04D0221C7C23393250
:1033000023701370231C4F33002101351970503482
:10331000052DEBD1214B2D22181C38300270181CC2
:1033200037300270A1209A705A7040005F221A5400
:103330001B481A54A320400019541A4908784978A8
:10334000385C014204D0191C533152330A701A7090
:103350000024211C381C0134FFF756FF0A2CF8D139
:10336000114D124E00242B786A78FB5C1A4201D072
:10337000315905E03059FEF7B1FC0D49091A0A31FF
:103380000C48043400F0F2FA0235242CEBD10A493F
:10339000084800F0EBFA0520F8BDC046A00C00106C
:1033A0004101000099010010A4000010B8000010B5
:1033B0009B010010E00D0010A0570000F0B585B093
:1033C0000190FDF715FB00226B4C6C4F0092161C10
:1033D000754275416A4A009B5D191368012B02D042
:1033E000022B02D15EE1654F02E0002B00D1CDE05F
:1033F000002303AA537023687F210B405C2B00D16C
:1034000098E02ADC382B00D18EE013DC072B6AD041
:1034100006DC022B00D193E0062B00D0B6E041E0A1
:10342000212B00D184E0232B00D187E01C2B00D07E
:10343000ACE081E04F2B4ED007DC3F2B62D0402B1D
:1034400062D0392B00D0A1E064E0542B76D05B2B06
:103450003FD0502B00D099E06AE0732B66D010DC8F
:10346000662B3AD005DC5E2B56D0622B00D08DE067
:1034700062E06F2B3BD0712B52D06D2B00D085E0DA
:103480002DE0792B4AD006DC762B4BD0772B3DD024
:10349000742B7BD146E07D2B23D07F2B25D07C2B3A
:1034A00074D135E031231370022E4BDD231C083B11
:1034B0001B681940542908D0032E43D0231C0C3B11
:1034C0001A687F231340542B3CD14C2203AB1A7053
:1034D00038E0322335E0332333E0342331E0352341
:1034E0002FE036232DE037232BE0382329E0392342
:1034F0001370062E26DD231F1B681940472323293E
:1035000020D11EE030231CE02D231AE0412318E0D7
:10351000422316E0432314E0442312E0452310E045
:1035200046230EE048230CE04C230AE0502308E039
:10353000522306E04F2304E0552302E04E2300E02F
:10354000492313703B1C03A8291C0022FDF744FBF0
:1035500023681A0605D5E91D0A4800223B1CFDF721
:103560003BFB2368DA0572D5E91D074800223B1CA6
:10357000FDF732FB6BE0C046300E00100800001073
:10358000A801001021430000A85700002368012271
:10359000134206D0A818C0B2002107220223FDF76B
:1035A000A5FA23680222134205D0A81DC0B200214B
:1035B0000623FDF79BFA236804210B4205D0A81DC2
:1035C000C0B202220623FDF791FA236808210B42BC
:1035D00005D0681CC0B207220223FDF787FA2368D2
:1035E000DA0606D5681CC0B2042102220623FDF7C4
:1035F0007DFA23689A0606D5681CC0B20021022213
:103600000623FDF773FA23685A0606D5681CC0B274
:10361000042107220223FDF769FA23681A0607D559
:10362000281C09300222C0B20821131CFDF75EFAE3
:103630002368DA050BD5EDB2281C0930C0B20B2186
:103640000A35FDF73DFAE8B20A21FDF739FA009B89
:1036500001360C33043400930B2E00D0B8E6124B25
:103660001B68002B05D0114800210922104BFDF7E3
:10367000B3FA104D104E114F0024019A2B78D35CF1
:103680006A781A4206D0A3009859E15D0922084BD6
:10369000FDF7A2FA01340235092CEED1FDF7B2F99B
:1036A00005B0F0BD064FA3E6D4010010AA570000F4
:1036B00014000010A4000010AC010010DC00001089
:1036C0000000001038B5FFF797FA002814D0062440
:1036D0000321201C00F0DEF80321C5B2201C00F0FD
:1036E0002FF9281CC9B2FDF7EBF9092C01D10B24E5
:1036F000EEE701340E2CEBDDFDF784F938BD000058
:1037000070B5041CFFF756FD201CFFF757FE0A4B4F
:103710001B78002B0ED0201CFFF7E4FD074CC823BC
:103720005B00074EE518211C301C5034FEF77EFA72
:10373000AC42F8D170BDC046B9030010A00C001017
:103740007F3A000000B589B000280ED0FDF71BF9C4
:1037500001A80921FEF75EFB684612300A21FEF738
:1037600059FB01A8FFF7CCFF08E0FDF714F9044B63
:103770001B78002B02D00348FEF758FA09B000BDB1
:10378000B9030010AC57000000B5FEE700B5FEE736
:1037900008B50A4B0A4A0B4903E010780132187049
:1037A00001338B42F9D3084B0849002201E01A701B
:1037B00001338B42FBD3FCF7B5FEFEE7000000109F
:1037C00005580000D0010010D00100105C0E001060
:1037D00002B4714649084900095C49008E4402BCA4
:1037E0007047C04603B47146490840004900095A71
:1037F00049008E4403BC7047002934D001230022C5
:1038000010B488422CD301242407A14204D281425F
:1038100002D209011B01F8E7E400A14204D281426F
:1038200002D249005B00F8E7884201D3401A1A43EC
:103830004C08A04202D3001B5C0822438C08A04223
:1038400002D3001B9C082243CC08A04202D3001BD9
:10385000DC082243002803D01B0901D00909E3E753
:10386000101C10BC7047002801D00020C04307B4D2
:10387000024802A14018029003BDC046D9000000D2
:103880000029F0D003B5FFF7B9FF0EBC4243891AF7
:103890001847C046002941D010B4041C4C40A4462F
:1038A00001230022002900D54942002800D54042CA
:1038B00088422CD301242407A14204D2814202D29F
:1038C00009011B01F8E7E400A14204D2814202D2BF
:1038D00049005B00F8E7884201D3401A1A434C08BC
:1038E000A04202D3001B5C0822438C08A04202D3F2
:1038F000001B9C082243CC08A04202D3001BDC081A
:103900002243002803D01B0901D00909E3E7101C5A
:103910006446002C00D5404210BC7047002806D0F9
:1039200003DB0020C043400801E08020000607B40C
:10393000024802A14018029003BDC04619000000D1
:103940000029EBD003B5FFF7A7FF0EBC4243891A4D
:103950001847C0467047C04600B5002905D000236F
:103960000139037001300029FAD100BDF8B5041CFB
:10397000A30719D1231C04CB0F4D104E50199043AF
:10398000021C201C32420FD1181C0B4F04CBD5193E
:103990009543354208D1181C074F04CBD5199543E0
:1039A0003542F1D000E001300378002BFBD1FEF767
:1039B0009EF9201CF8BDC046FFFEFEFE8080808080
:1039C0002578000D0A413A2000202025633A200086
:1039D0000D0A4D3A20002020473A20253032780D3C
:1039E0000A0025732025730D0A00444D3130005321
:1039F000455249414C20434F4E534F4C4500726550
:103A0000616479000D0A4279652E2E2E0D0A004C54
:103A100043443A25303269202D2025690025732042
:103A20002573202025694D485A0056313300202047
:103A300025692E2530336956007475726E656420D1
:103A40006F6E004241543A2025696D560D0A000DF3
:103A50000A2530327820200057616974696E67202A
:103A6000666F7220646174612E2E2E0D0A00426111
:103A700064206D6F64656C0D0A00526561642025D9
:103A8000730D0A004F4B004641494C4544006F6698
:103A900066004C43442064656275672025730D0AF7
:103AA00000000000005C000C000C7C287C7C447C46
:103AB000241048285408000C0038440044380020E2
:103AC0001008103810804000101010004000201026
:103AD00008384438007C006454484454281C107C46
:103AE0004C542438542004740C28542808543800AA
:103AF00050008050001028442828284428100454DE
:103B000008384C5C7814787C54283844447C443819
:103B10007C54447C14043844347C107C007C0020A9
:103B2000403C7C106C7C40407C087C7C047C7C4469
:103B30007C7C14083844787C1468485424047C0441
:103B40007C407C3C403C7C207C6C106C1C601C6489
:103B5000544C7C4400081020447C000804088080F9
:103B6000800408007844780007080400000000BFC3
:103B700001BF010905000007000700070007130A3D
:103B800000002000E400FC003F00E700FC003F00D4
:103B90002700040F0800000C011E01FF03FF032291
:103BA00001E201C2190D00000E001F001101910178
:103BB000FF007E00FC00FE0113011101F001E01482
:103BC0000A0000EE00FF0111011101BF01EE00E04B
:103BD0000130011001050300000F000F0A0500006D
:103BE000F800FE03070701040B06000000000104B3
:103BF0000707FE03F80F08000000000A000E001F70
:103C0000001F000E000A1109000010001000100033
:103C1000FE00FE00100010001008040000000480E8
:103C20000780030D070000100010001000100010A6
:103C30000010080400000000800180010D07000C46
:103C4000000FC003F0003C000F00030F080000FE4F
:103C500000FF01010101010101FF01FE1008000048
:103C6000000002010201FF01FF0100010001100834
:103C700000008601C7016101210131011F010E0110
:103C80000F08000082008301110111011101FF01E1
:103C9000EE11090000300038002C002600FF01FF63
:103CA000012000200F08000080009F011F0111016A
:103CB0001101F101E10F080000FC00FE010B0109F8
:103CC000010901F901F00F08000001000100C10124
:103CD000F1013D000F00030F080000EE00FF01118D
:103CE0000111011101FF01EE0F0800001E003F014C
:103CF00021012101A101FF007E0804000000008CC9
:103D0000018C010804000000048C078C03120900D8
:103D100000200070005000D80088008C01040104CD
:103D200001110900004800480048004800480048C8
:103D30000048004811090000040104018C018800BA
:103D4000D80050007000200D07000002000300B1F1
:103D500001B9010F0006190D0000F800FC0106036F
:103D6000FB06FD0505050505FD05FF050601FC0132
:103D7000F8120900008001F0017C004F004F007C28
:103D800000F00180010F080000FF01FF0111011187
:103D9000011F01FE01E0110900007C00FE0083010B
:103DA00001010101010183018211090000FF01FFEE
:103DB000010101010101018301FE007C10080000E6
:103DC000FF01FF01110111011101110111010F0882
:103DD0000000FF01FF01110011001100110001128C
:103DE0000900007C00FE008301010121012101E3A3
:103DF00001E20112090000FF01FF01100010001094
:103E0000001000FF01FF010A0500000101FF01FF92
:103E10000101010B060001000101010101FF01FF89
:103E200010080000FF01FF0138006C00C60083018C
:103E3000010110080000FF01FF0100010001000165
:103E400000010001160B0000FF01FF010F003C0004
:103E5000F000F0003C000F00FF01FF01120900001C
:103E6000FF01FF010F001C007000E001FF01FF01D6
:103E7000130A00007C00FE00830101010101010121
:103E80008301FE007C0F080000FF01FF01210021DB
:103E90000021003F001E140A00007C00FE00830188
:103EA0000101010101038307FE047C0412090000E3
:103EB000FF01FF01210021007100DF008E010001E0
:103EC000110900008E009F01110111011101110162
:103ED000F301E211090000010001000100FF01FFF0
:103EE000010100010001110900007F00FF008001B5
:103EF000000100018001FF007F1109000007001F81
:103F0000007800E001E00178001F0007190D0000B3
:103F10000F007F00F001E0017C001F001F007C000B
:103F2000E001F0017F000F120900008301C7016C5E
:103F300000380038006C00C701830111090000013E
:103F40000007001E00F801F8011E00070001120919
:103F500000008101C1016101310119010D01070159
:103F600003010004040200007F01090500000700AE
:103F700000000000070B064400FF0144004400FF5E
:103F800001440B0600008C001201FF032201C40D46
:103F900007820045002500920048014401820C067A
:103FA0000000E60019012601C000200107040000FE
:103FB0000000010002080400000000FE01010208E8
:103FC00004000000000102FE010B06000088005002
:103FD0000020005000880B06000020002000F800A0
:103FE00020002006030000000400020B0600002051
:103FF0000020002000200020060300000000000137
:1040000009050000800160001800060B060000FE94
:1040100000010101010101FE08040000020002008C
:10402000FF010C06000082014101210111010E0176
:104030000B0600008200010111011101EE0B0600C8
:1040400000600058004600FF01400B0600009F0082
:10405000090109010901F10B060000FE001101111F
:10406000011101E20B0600000100C10131000D0049
:10407000030B060000EE00110111011101EE0B0609
:1040800000008E00110111011101FE080400000062
:10409000008C018C01080400000000000208010AE5
:1040A00005000020005000880004010B06000050AD
:1040B0000050005000500050090500000401880025
:1040C0005000200B06000002000100610111000EEB
:1040D0000D077800860132014902390242027C0E46
:1040E00007800170004C0043004C00700080010B01
:1040F000060000FF01110111011101EE0B06FE0087
:104100000101010101010101820B06FF0101010111
:1041100001010182007C0C060000FF011101110168
:10412000110101010B060000FF0111001100110037
:10413000010C06FE000101010111019100F2010CC8
:1041400006FF011000100010001000FF010804001D
:104150000000000000FF010704C00000010001FF93
:104160000E070000FF01180024004200810000013A
:104170000C060000FF0100010001000100010E0714
:10418000FF010C003000C00030000C00FF010C06E5
:10419000FF01060018002000C000FF010B06FE0012
:1041A0000101010101010101FE0B06FF01110011D6
:1041B00000110011000E0C06FE0001010101410179
:1041C0008101FE020C06FF011100110011002900FF
:1041D000C6010B0600008E00110111011101E20B56
:1041E00006000001000100FF010100010B06FF00B5
:1041F0000001000100010001FF0D0703001C006029
:1042000000800160001C00030D071F00600080019A
:104210007C00800160001F0E07830144002800100D
:10422000002800440083010D07030004000800F08B
:104230000108000400030E07810141012101110161
:1042400009010501030100070008000A0100181117
:1042500010133831303378717073C8C1C0C388818E
:10426000808384848782C5C4C7C2757477723534ED
:104270003732151417120207020802010003010960
:10428000030402040205030500062024282C383C00
:104290004044484C4669726D776172652025735FB2
:1042A0005631330D0A00252D3130732025732573C7
:1042B000000D0A5479706520273C636F6D6D616E47
:1042C000643E203F2720666F7220706172616D73BB
:1042D0000D0A00557074696D65202575730D0A000F
:1042E0003F0025730D0A0D0A00564F5941474552AC
:1042F000203E3E200025630048656C70004E6F2014
:10430000706172616D73004B6579207072657373B3
:10431000003C6B6579313E203C6B6579323E202E46
:104320002E2E0044756D70206D656D6F7279006C76
:10433000004C6F6164206D656D6F7279007400547C
:104340006F67676C6520646973706C6179206F7545
:104350007470757420746F20636F6E736F6C65007A
:1043600062005265616420626174746572792076BE
:104370006F6C74616765000000800150008002501E
:1043800000800350FC3F0150FC3F0250FC3F0350B3
:1043900022B8A60AEFC4552FAB2AAF953FD3383ABF
:1043A000E5E966B07B7FAB8C67B76BFE3B3C2B9837
:1043B00067BC59AC68C4E7E8D6121380934569D04E
:1043C0006958880F92D161EB85C332D86BF36228AC
:1043D000B27A9A52B58E6AFCA2746CCE3A85A61651
:1043E0002D00086472B9286FE1796CFA37F4D7F8B8
:1043F0003383E97E18841242144F88AAE376107D35
:104400007E2070CC7D4A33CB680E2B2C48544CCC8C
:10441000AC174B71AA4EDA9F73C24AE61FC76B9E58
:10442000EBD541207A2F8ED5C9456A026E5CE10F2B
:10443000148F29FD5788D9ABFA2CF0E840B539F82C
:10444000D0D0AE6B16431F6D41AE3EC2524D6D5C77
:10445000A55E65820688A59F175410EE2E7DA4D117
:1044600003BC4EE001D569E088582D875FA29C20EF
:10447000D638E4298843FC9F09D5FB80F2097A836A
:104480006D2D2B2BF94BAB29B56303BAA7299AB82D
:104490008B0489BBA3C63A5100FDEF7A7AC910FCA0
:1044A000265417315F2093A24F486D5BC49F7471EF
:1044B00035CCEB21B21D6345EAC0A2D84A220E8F4B
:1044C000BEFDBA596C82699EA4D703E86A6443A30F
:1044D000C6F5AC34701A2FD445A1B80D88E830CC9D
:1044E000215FE753006AFA7A1371E2C3A4C4938A86
:1044F000572D44AEA1CA43CCAB7904CEDA775988A4
:10450000629ABC0259FD9ED1E0B649D3511A992B4B
:104510003ACDD5A12E020088B2889D2F104916945D
:10452000E656CA2DF6741183ABA14411CAD59EBBC1
:10453000812D809EBA4291CDD8242D486DCEA68083
:1045400015215ED28A48A57EB28907BD0ACDC16019
:10455000E39294FD0787E5DF1728603F34493F4128
:10456000BBDB29B4D91C2E3BFA03B45D1B02DB4D27
:104570004E5CF1435CF1419D3BE10C64CA1A51DA97
:10458000D59ACCDD2AC2182416805A901730BF1253
:104590009F1C8E3EF3B0EB037859A1CEB636DADC21
:1045A000B65D7AB06239F624028E1893AAE3CD86FE
:1045B0009DDFA3BAA1D33A5D7277E39B7A5E524541
:1045C0002FAC45268FE7E418A1957D45DF92148036
:1045D000AC479251976315C544E2DFEB57618149BF
:1045E0004E07ACDFFCFB535C4BC0669EECC4C0FFC7
:1045F0000F8330754BDAD2AC81E493DEC9998D24F8
:10460000F490D248BE21C43B57ACC44ABBAD585D00
:104610005F676181321BFB8B0EE287F547EBD05D54
:10462000E12D5C14189CAFDF220CE8905BEAFB885C
:1046300041F02B1587771A716AADA54CECCDF6B118
:10464000E13CC7CDD3C232A23565999A396FB21910
:104650008A2A4232360EE841C90A730C4A41E2B056
:10466000A19FEB70375FF456C8831E410BE02E3FCD
:104670000AECA79C4FA01711F03117DAC128E9BC4A
:104680002BAB39B33A773D1DC990221928860A9180
:104690002A2C3E863805C3C58F82AB27F33AECEE51
:1046A0008E41B29567B036E6DB442C3CEB469FA8C2
:1046B0008A806C156AC15C2B98D9381EF70BAD7FC8
:1046C000592DC2EE6AB38C2BAD0572E4B8DCF27AD8
:1046D0005C2AFC2A35F1CE3C6D4994A2D273886FD6
:1046E000DFFB1A6CA61A3E25FCCAEF81C2D3F61C6A
:1046F00073956F9BFA591BD2F40C20B752A826A1D0
:10470000EF0BC3C27F0DE12DE8386E3512391B3532
:104710001A34AC08D8FC9BEAF885C9E66309FF8522
:104720005F7969472625C3CDD53DE5A3EC4E1266DA
:10473000268693C95822505FB91EB40BEAA83D30B3
:104740001CB1F1EBB721A4707DA7A7CC6B5D23A7AB
:104750009FD613A932CD48F0FD37D6F419E223B025
:1047600067A1F2350CAAAA855CB3176F39B54A4C1C
:10477000788D74D3ABAC2C86A423813D480834C516
:104780003B0D89B395DAF5A6F66FA110FC79673B6E
:10479000757E1A8089770BE910ABA9CE20A5D6D2F9
:1047A000FD27EDD9DB85DBA2ACB882368A666A5A72
:1047B000BCC89309DFA4001DF4DAD5ECDB155D134A
:1047C0000FC569B77ACCF573ACFFCBE4AB221EAB57
:1047D0007A909E37229096C51B7D7934330043171B
:1047E00020BCEF0EAF9C1C688256140F01A04191B3
:1047F000E10D21CD17F329883481062FB9A740F0A8
:104800009F00C699F916AA1C28FDE3E8D45145D5A6
:104810004FC4222209CDC34EBDDC9DD78F5540EE3B
:10482000455B3609B3C2E2544FFC2D80E151582557
:10483000A7AFE4BD84BA0DD554B198B671CC0CD3F2
:1048400073FD9FF776829B8AF58E656C91F51EABA2
:10485000A6456183C2AB3BBCCE52F14BF7C2E70C1D
:10486000EDF71AD97BC88A9C11511F128FA3EBDA7E
:10487000B80E940EA1AD9523EF594B1FCAF84916F7
:104880000C49A946A87280BF8EDD45490FB446BECB
:10489000075E3F3FBBF079067C9D4F99D59056BC93
:1048A00030D2C9FACDDC1B12E26DF217612B1AA7C8
:1048B000D45DAFAC50E2A05C1A6B32C15207875E88
:1048C00095C928BD7BD13B7A59B9180DFF5CA0353D
:1048D0001074BC558E1C27CA809129D982A3A2ECE2
:1048E000C8F8B1C12BA2A2C356548BAFF6BB9DCE64
:1048F000077CCFDC13B2CF1A69B8C402A25DC1BE77
:10490000F2CDBA52863A9F77752275443311E3C2CD
:10491000318EC3EF94B7852DC3406D413487491F55
:10492000F4C503E199B8113E9AB826CB7D8BF7B553
:1049300027CA308A30605191E0936D87A5AA780527
:10494000BF0E3363AD2437C2E407F133A9A6B78B9A
:10495000090CC477A1FD8EF8CEE4186D230862AF70
:104960009AC0700E88270E5E39985423B979875003
:104970003EB9FF1D443FA9754A3E078A9DB237FFE5
:10498000A4A68F7C76BBB7F0E8E5B8C67ADA2E909D
:1049900018B2247012640786AF07BABC7BA230A19C
:1049A0008FBA2F98B178576CB38ED1D62FA2FBBB9C
:1049B000DB7245DBA8CE1BAA2E553E70A0CFA7BE4A
:1049C000E2ECBA95266561B8A6FF0B13D2E72FB8C3
:1049D0007B43920CC3AD7774189784678A05FBA15B
:1049E000FE5098B54842109CC7000004A3D50ECBDA
:1049F000B4990FD96D241036E5CED12DD07314A8FB
:104A0000937AD310AE44D39CC9A5B7DB1363766801
:104A100018D8FABE2987410BDF7420D69136497C1D
:104A2000E85DB3DC2957F71CC05CD92380035F71B4
:104A3000B8BC260251C06DA780EB2F0ECF63FA3CA5
:104A4000B279D702080F2965536BCE5FEE1E13486B
:104A50000F4A4A655C2A7D691E1426BB97F74F22D0
:104A60008E45F3B31AB6AC4157C966360CA358BD90
:104A7000243F2E25085AC5908BC97EE3E86117783C
:104A8000C3CAD20304D8748314AFBF5A8027BFA10E
:104A9000D4E492F8503913DFFBBBFB5626C1BD9915
:104AA000F61E4C943579675F27D7C43B8AC9C62B5D
:104AB000EDA8DA7D9638C8BF9E587FD360C4C2F295
:104AC000A1005C23C3C5FAF3C7C4EA1FA94B86DA69
:104AD00041DCBA0CBEF663F6D13746A8CDDFD54E21
:104AE000119CBC68104FDA592270F725445ECE4401
:104AF00092295289B9E68B6DFF403E94D186A82851
:104B00004677E5F5ADED31AF047429CD691AA57E80
:104B1000DB08C23AF041EFB690789BB46B9B10F57E
:104B20001A0CC6F791EE2E370CA0897CC6C57854B6
:104B300048E5025BB73EEE61404A3C834F79BECA0E
:104B4000566D929FE3200EB1C34D8F0FC332702B71
:104B500085FB9740EBEF7C1D52EEAE2FE12AF2B8B9
:104B6000E5266ACDE624BB2832BF81B5622240CC5F
:104B700004635A9F5FA96C2DB0A3D1268BBCF8BBF0
:104B8000DC26188B8BBB37AEA9C9A20AD4848C8BC8
:104B900026C164DBF62422554541E65A2A0D9B12B4
:104BA000479C7ED9423B7C7FB373A190C68187B07E
:104BB000CA90C7E3C243B7B8BD1E3C477F197A0508
:104BC000F7F1BE171A0B9C9CF80021BC287F9C5E55
:104BD000F45360B6A68A554FC640F1A05743B5B905
:104BE000A660E371501EB356312D6184C62D06FEBA
:104BF000B695C6F594D67983C0481AB44385C64B9A
:104C0000B576721EDBB6462CDDD31C00FF4B48BBCD
:104C100065A72681C10C05C57B64B96029B814D984
:104C20000FED59B1A7856978AB9E12398E75922C1C
:104C3000CF7793808FDC3BDCE88ECFAE998DEBC9CC
:104C40007867690F20B67DEB46BE02FAE8248D8AAC
:104C50000789BD9D82FB324B560B62EA1C4659B553
:104C60005C03B092CAAE633C4DB9F824EF8D47980F
:104C700057E81E8F6FA5CEF50FF5F4ED625735F0AE
:104C80002892F93192DA60F50190C49C4E402B20B5
:104C9000884C0B6A2029962187A38640D4B0C9444A
:104CA000C701BF18CFE5237B6CD191C00C8533C2FF
:104CB00033F3DF1D2F4178B49852C7D34AA106A918
:104CC0009A5FC58672CF475CA4FD82F2F07EB21E69
:104CD000F0DA2D6E030A3F2BF6FE080C3D2DACE8F2
:104CE000E5B36381DB65639E9A4CB478B70F589D3A
:104CF000373CD4D3C479122D9E9B0312A36E29187E
:104D00003D774969FD50EDB830C2FF055FF5EFB55D
:104D1000963615582B39A428986894D50D3CA68B47
:104D2000B6DB4ACE001FB19198C29E9119D5299C3D
:104D300085ADE7549E63FB18E1BC1129DD7D860338
:104D400028CBB4CFD2D21C264FD03A5E70A30D4DE3
:104D5000D4F748BC988A8FA068A8DA3A5C858F7A25
:104D6000A1C00C0EDFE95C5714744C936E01515EC8
:104D700061167DD34C330FAA69EFA0B4330680AC23
:104D800085FAB44C3255AC8AF84E8B1DCF14E8E549
:104D90009AF55CEE96A24D852A964EDA6920262772
:104DA0000ACB99FA9BB3EA6748B5A0B0D5D494561C
:104DB0007C77A9AD401260F14A258152DEA80F8BA5
:104DC00037DEF88F187125A3CF0DEFC59B6BD0741C
:104DD000E712EA46914B592F5B9D39E4E510C5284F
:104DE0000EB57689A07CE36C0C2C3DFF70D8430E89
:104DF0006DB782144F55D2655684D827BF4F14140F
:104E0000108483B87158AA0737E7364665E856B864
:104E1000DE16606681921F9B321D1C244950A661DC
:104E2000AF276173DC2D2B4FD39E1345D8DFF5736D
:104E3000A54A00053C5031A600012E7DA044A08665
:104E4000BEA2A38D30DDFF70C56429C84FA09912A2
:104E5000D44A62243D53C5B1476680903AF1EE339F
:104E600035A17C2C60F0992178BC5B68F8E4B27ABB
:104E700008C4884DB54F5068E8269EEBC9E1953AC5
:104E80004F41D004E1D62828237D71F37BDD2EA885
:104E90006AF9FFB62EB825640DBF47A0BEAAC74267
:104EA0008F755B79B2330EAE12725DEC0D51B49119
:104EB000B5E0FBC936FA97F3395FE430F5A2586ED6
:104EC000A173185BBCF36B3100AC81D70499A8EBDC
:104ED000ADECEC927AC632DD5239F5D6B7EBA1EBE8
:104EE000E824D7AF7889F6DFEF28DC8B0306BF080C
:104EF0004F2490077159E5025AC8232BD508397001
:104F000097A84ADC1CA7F75ED389FFCA29A3DC381F
:104F1000DC299148B87E231008F6C6E15706BF2861
:104F2000DAE96367A248E0447D48406C20143BDD29
:104F30009FB7447FB55CE0264F4CEF9F69CCF31DD3
:104F40002A0D7CAC4310BB788773D46B8CD6829CC3
:104F5000FB4FE35B4C0F7804199A23CB9B6A3FE12C
:104F6000C938AAAE9DF8E7F010E3B3EFB05440AEF5
:104F7000A9FE6AC07D6839D42BFF0D8912A4C96DC2
:104F8000F04DDBA9CDD38E453059377AD87AB18828
:104F9000BDE883786F3D8152BC7D357DE8A9AD9336
:104FA00035FFE8FCE4B3FF843A798B5F162A8CF571
:104FB000BE98426AE4E7EA164575E616DF18B8CCF3
:104FC000345DB2B7CE78F4E980DFC61C343458B90A
:104FD00076EFED8B56E4ACA906941C7AF16F2D3672
:104FE000080854C286845678258A7D18619284CE3A
:104FF000675DE36D62BD7668C721DFD321CC59952B
:10500000D92048F338EE3114DC0E2F470FA70EF0ED
:10501000D136C8655312621D3AE9AE3D7DD2FE100D
:105020005985B14B65ECDB3AE0D68D8AFEA2212290
:105030003DE5BCB9138B63DE929ECB4D8545F4CF25
:105040000D8160E9E3CA9B3644F84F7B0BCC7D6849
:10505000F0BC512192CC6B67462E5A04903A9A6D5F
:105060000F18CB35077A51ADDC59C2F5390A2E1825
:10507000AA8F8DF6B1F23AF49EB671B8FDAC8133C9
:10508000A2B0B897C0886E52CBC5B262D31C0FD203
:10509000EB8F268D449B4448C175BFA67252609425
:1050A0009F0505A10D1C9114A764CF7EB327ED6A5F
:1050B000655321A01632753041BD9FD400CDCA99E9
:1050C0007599F8E51AF23BC26AF858C755C8C96025
:1050D000BBE96E607C78CED97F6D87D7A8AB02C85C
:1050E000729F3AE22F5122A2211FCC331913E9E417
:1050F0003DAA9E87AC6CE19744F384485E2A503009
:105100005085DFE3A3435016CB9465E159756DECF0
:10511000E31AFA959101FC3F5E4C150A764F9FFA0F
:10512000E3430AD40DB140BBF577BD03FD2AF88BEC
:10513000A683740C5A06D3EF1C0F34B9599990CF3B
:1051400058AB84EACB4708578A9BE97EB9F553C828
:10515000B816F2F7E96D00EB202CEE16CDCBF2433A
:10516000ECBD5FCFA7561722FEDD4FBEB3A52F8E35
:105170008CA837496282436B173A6A12BBE3BCDBE7
:10518000BD4DBC74BFA57DBB1B35B01B7D44E4F396
:105190009F74FC60718D5D362769134DCDA3AC36CD
:1051A00049FC7D0C84EF53C0F4CD7190B52C17C22F
:1051B000BB32FA467363BF7B4E8E9A0A6B02ADB95F
:1051C0002E639C5EBF3660A7B3A99715A78154E0F4
:1051D000235521DB40BC222F51F65DBEB7571CEE94
:1051E0004ED3352E333B12864C9BB30BA40288FD65
:1051F000D4FC2390D28F0577607BDD864A2C8A9978
:10520000ED7533079F7B46E420F4C1D52D662175EB
:10521000AE20E5797DCA7CC8FA93271E5F4E39E13E
:105220009F6A2DDC04BB75D7286E5AA98C0E68E8DE
:1052300027D308546A6DA2D5594B5B8D91F057283E
:1052400004D2E6198A4C25C237F9B226B645C4A85D
:10525000D5507CDD1C397E752B6078E574966CF238
:10526000F3D5A93C8FF505B8DC215D4BEA3BA4AD35
:1052700043B02F616364D71C5D4FF679F268C1CCEF
:1052800085A765BF3F9A43CC20AB5A64C4EE8068C3
:105290000D0F5BEB56CEF52816D5AC8A15CE685EA1
:1052A0001BB1DA2110FA1B280FE3DEC3B351191327
:1052B00082E6D6A735B51F081A98C2CC9EBD3AD54E
:1052C00084D4C0945DBDBB0BB36E5BD1577B640EC1
:1052D0001DB81C35B14F6A456FF703304156E7EBF7
:1052E00016CF84EB6388A3248FAD37FB9CB9D459C8
:1052F00086942165C76DCA64EF7B2B5DB483D30AA6
:105300009C5AF4D517DFEA05D182789F2B364B8B58
:10531000C884348AD0EEB95E080F2F2D59F4AA2C18
:105320008D9B95946CD97F40B73810B55FBF2D89A0
:105330002D7BF8188A2AE746D99CC832DB63079F81
:10534000F39E3C5CD60DCC207B1C1A35A93324334C
:10535000ECB22BC182EB1EC55CDFFF357682188E66
:105360005327533F6653FC867923CB386D1F218129
:105370004FA28E66D95F4AC3E94A7BC36B80B53CB6
:10538000EBB01FD05B7B68CD4D123145701F1714F9
:10539000BFC8C71522D9222FE2F543D44618B974E5
:1053A000FFC0FED263761CA7FC866B7C3311651DA3
:1053B00076EFA0AF59120DD5FCE703B47D8D934F66
:1053C000C91B1F73AFA91AEE56E8F19CF90B738F36
:1053D000B9884D3D8FCECCB0B5952044C12F5BB67A
:1053E000592452AB85917980DB19749138C70AA58D
:1053F0000A1906488BF5B1AE3D512D151F92B02903
:10540000B140BD34FBBA1A2CCBCB93D58DD8B32188
:10541000751440B288087186CB8F4942CAFBC2A678
:105420008936EB5DC27E076706D8F5EFF165DF834D
:10543000F76186C33C2433841F8942462A93A9BF5F
:10544000267C4F355D0C8A58DE553B15843C15682B
:10545000B54245A7CA7858B1516C6FB1BB5E181FF1
:1054600092AC091AA6C8858055028F846310C37C4C
:10547000A64526B8A95E201BC6B859F2C6889C98D6
:10548000418A789C5FF48F19773A064BF2615AD4BF
:105490009CBA886948AD928EF94ECB6C722A29DD90
:1054A00030D8E587D3BF73EEABAE0F1E1703828FE4
:1054B000157A27667305614ECE4CAFB3543735B5B8
:1054C0002A1D5513033D3E2A56FA22BC30438BA5B4
:1054D000AD6955E72AA2B27449398519F844BF3538
:1054E000538DB9B1A2B9DD44D2A73E9D922CC3F42D
:1054F0003702FF4F99962580FEC1493AF92A307646
:105500005E618B6A8344245B821B6B86536C7105DE
:1055100074EFEFC8A3F3A16F124FB158E26FDF4AE7
:10552000B344FC716DBACB8377FD053643060C7727
:105530000B458AE08C7412C744D176ED7E3F8748D4
:105540001A9CA8ACFF86B71890F7FCB80B5AAFF6B8
:10555000895425E30F0D2FFC83E9441D4F532D0D76
:10556000EE930D7C47733A4E853F5A324942A9A8C3
:1055700036DAFA33A0AEFF6A90C3BCB9766160CD6B
:105580007788CD72AB0CC20B1165BB45CE53686BEF
:10559000D2E2A94ECC5FCFC8B9F9177892E5AC3DFD
:1055A00072518FA42D505FAE4D2E455B99911EC553
:1055B00060B5E479AB8C607672010BC7957211B956
:1055C0005CD9B5096B4A1871519B28DCA480CCA129
:1055D0003C7A4647842F133A8D58D2042805115F30
:1055E00027BEB6F1883EF6D0FEF9076BB78A48842D
:1055F000390FF0BDE0BDB5B61AE78EA68DDF3EF8D7
:10560000DEE78AF8526B7CA88EB0BB1519895B94D3
:10561000EA46EC048F8D730DD6F9FCCC88424250DB
:105620005BFAC0B05287DD28F7287D06EB57313989
:10563000F5DC25A82C47451117128356449326AF55
:1056400076BB02066B4BB8CF1DB3E9A7F9B6C54DC3
:10565000E63C48BEC5DC394CA4A738061DBD43CC8A
:10566000CD809A6067CA1BE15B83B768C723F7DF09
:10567000821E057DCB45701940D03364D0339D9296
:10568000F2C5851906FB3D3015324C9F97AC9CEE58
:1056900006BA3C1BC12077AAF8C3160C369935BA56
:1056A000B439E3C9E39BD6711CEB0289AAE263B962
:1056B00027979F1F8E540C8B34CFD8F76E90DEB790
:1056C0002101E9B1E9E5AC5679E44C4CACF1A4E137
:1056D000D79E2F4ECAEFACA218EBAF4CFEB001B96B
:1056E000B5E9EF6D26DD6613D07CF5FBBA1EEE281A
:1056F000E8208633AA85698CDA22B0BEE48658CFCA
:105700006BCDE3BA92C4ECED958C291A6F990C9F7E
:105710003926C314BD2F497999164058ABDB4C810B
:1057200087E5276293EB67BD76144A97FAE6A002F5
:10573000C153FE7371DC350E21C3754DE6BFFB24EA
:10574000A475B29C37D6B1BCA2D1911B82879CECC8
:1057500029098A7F621875E1FB8F6322843CEDDFA3
:1057600027347459D38EECCBEE099E139317CBBF1D
:10577000002E6C014D9CC1D6D0012E40926BC815F5
:105780007A7A897D97FF71016C1EFF090744CC9BD3
:105790000304050A08060BFF0209070D010C00FFB0
:1057A000202020205F5F7C002C0061004469737022
:1057B000206F66660D0A00555345520046004700AB
:1057C000424547494E0052414400442E4D59004342
:1057D000005052474D00555345522020200066206E
:1057E000200067202000424547494E2020202020ED
:1057F0000052414420202000442E4D5920202000FA
:1058000043202020000D0C205A673B00000D0C2087
:105810005A623F00000500000003072061A13A0022
:1058200000FFFFFFFF4D000000E04200000000000D
:105830000059100000F8420000FD420000FB420049
:1058400000FF000000310800000743000011430082
:1058500000AF42000000000000510600002343009A
:1058600000FD4200002F43000000000000F1060090
:105870000031430000FD4200003D430000000000F5
:1058800000890800003F430000FD42000060430023
:1058900000000000001906000062430000FD420005
:1058A000000F000000F40100001A041B041204138E
:1058B00001010402010204030404040000D657009D
:1058C00000DE570000E2570000E6570000BE570018
:1058D00000F1570000F857000000580000D15700B1
:1058E00000081C242C4448586C741808180219022B
:1058F00019081901180418011A021A0111081102D5
:1059000012021A081201110411011B021B011002DC
:105910000F0810081B08100410010F0414021401D2
:1059200015021408150812081504150114041602AE
:105930001601170216081708130217041701160498
:10594000130813040D020C080D0801080D040D01C5
:105950000C040C020C010B020A080B0802020B04D7
:105960000B010A040A020A010902080809080208D0
:1059700009040901080404020401070807020802D7
:1059800003080801070407010302030106020508D2
:1059900006080408060406010504050205011904A9
:1059A00020202020202020202020000000010000B6
:1059B00000B7570000BC570000BE570000C057009A
:1059C00000BE570000C6570000CA570000CF57005E
:0559D00000D1570000AA
:00000001FF
